:020000020000FC
:1000000066C71B35E6B2F5BA18950F93FFD408B74B
:1000100001FFFCCF02E008BF0F910A95B1F70895E8
:100020001DE00FEF1BBB94989698969A949A0BBB81
:100030009698969A08951BBB94989698969A949A37
:10004000DABB95980000000009B3959ACABA0895E2
:10005000222339F02F93EFDF0D9313952A95D9F7CB
:100060002F910895222339F02F930D91DBDF139503
:100070002A95D9F72F91089515E0DDDF0860D2DFCA
:100080000F9302E3C2DF0F91077FCCDFC9CF1FE0E0
:100090000EEAC8DF1EE000EEC5DFC2CF97981DE074
:1000A00000E4C0DFC8DF06FF06C002E0AEDF979ABB
:1000B00006ECABDF08950AE0A8DFBDDF06FDF5CF53
:1000C0000F934AD541747461636820000F9107FF54
:1000D00061600EEA60FD0EEE1FE0A4DF08E060FD47
:1000E00008E215E09FDF02E390DF01E060FD01E23E
:1000F00099DF0AE08ADF626010E001E093DF09E146
:1001000084DF8EDF60FD05C027D546756C6C00006E
:1001100003C022D54C6F77001FD52D5370656564E1
:100120000000089500E410811027108330270895FF
:1001300010E198DF07E236FD0064089534FFF2DF36
:10014000821B9D0B089514E076DF0F93201B28F48B
:10015000022F79D401E269D4222710E179DFEEDFA2
:100160000F9119F0013008F01894089508E5EF9305
:10017000FF932F933F935F9352E30081220F285FF9
:10018000E20FFD1F308135FD3F7E3F7707FD306870
:100190000F7714E047DF218182179D0708F4282F8D
:1001A000032F0F70042B13E03DDF00E111E03ADF75
:1001B000022F12E037DF03E2403909F0B9DF60FDBA
:1001C00012C0403D89F0523379F4122F185F0F921C
:1001D0001F920F9308E2019F1FE02DDF01150F9181
:1001E0001F900F9008F00F7D37FD006834FD00610F
:1001F0000F9316DF0F9110E015DF08D41DE01BDF11
:10020000102F1076C1F400FFF8CF1DE001E00ADFE7
:1002100013E011DF00FF20C0403949F434FD05C070
:1002200002950695032706FD07C08DDF01C086DF16
:1002300021F588940BC000E10F930CE3F6D30F91E6
:100240000F9301D40EE3F1D30F9108945F913F9186
:100250002F91FF91EF910895403911F0A21BBD0B32
:10026000132F1F7049F706FD02C002FFE5CF5A9514
:1002700019F3513011F402E7D8D38DCF4F93AF93D8
:10028000BF93D0872227AF93BF93B0E0A0E63C9105
:100290003078306190E088E040ED68DF9E918E918B
:1002A000BF91AF9190F0082F092B40E929F0432F1F
:1002B0005DDF58F040E843278F939F9390E080E004
:1002C00000E4008753DF9F918F910F9305E608F4B8
:1002D00006E60F91BF91AF914F9108954F9345E07E
:1002E000CDDF18F44A9504FFD9F74F9100F5202F80
:1002F000EF93FF9331D44550302D5472616E736685
:1003000065720000C0E618E08FD309919CD31A955E
:10031000D9F722D4204665686C6572204B6F6465FE
:100320002000022F90D38BD3FF91EF91022F0895DD
:1003300000273327C0E609931993299300270993CF
:100340003993099309930993C9CF2F9315E0F0DFEF
:100350002F9128F01081122B108302E056DE0895B1
:1003600000E816E040E050E0B2E0A0E0C0E609930B
:100370001993299339934993599389939993AEDFAC
:1003800008950D911D91153079F40D911D911295DF
:10039000012B00830D911D91112311F4003F08F0F2
:1003A00000EF01830D911894089566DE02E32DDEBF
:1003B000D3D32C20456E756D20002224F0E0EAEAAC
:1003C000239400E401873324222731E090E088E081
:1003D000C7DFD0F104E629D314960D9101830D9166
:1003E00002830D9103830D910187222DAEDF60F111
:1003F00001E61BD3222731E090E082E1B1DF20F15A
:1004000004E613D351964C90232D32E092E080E025
:10041000A7DFD0F003E609D30D910930A9F40D91BF
:10042000023091F48827992712966D900D910483DC
:10043000139677240D911D91143071F033944A94E2
:1004400019F7F2D28894089587D34665686C65726F
:100450002100F5D208940895082F092B71F0AF936D
:10046000BF93EF93FF93DC010AE01D9111930A956E
:10047000E1F7FF91EF91BF91AF91CF010D9105830E
:100480000D9106835D9057820D91002309F0018341
:100490000D91002309F002830D91002309F00383DD
:1004A0000D913A96552029F06CDF41F632965A9418
:1004B000D9F7C0CF0781000F065FE00FFD1F008155
:1004C000013048F001810117A9F70281021791F765
:1004D0000381031779F7089507813896222706C00C
:1004E0002395329610811327107B21F00217C1F754
:1004F000222708940895CF0130E2EEDF20936A00AE
:1005000028F1218129D32C2042756C6B2D4F7574F5
:100510002800022FB0D209E288D2FC0130EADCDFE9
:1005200020936B0058F0218117D32B42756C6B2DF3
:10053000496E2800022F9FD209E277D20DD32065A1
:100540006E746465636B7400FC018894089519E00F
:100550002481EEDE98F001E01BE026813581EADEA1
:1005600068F42681D21750F0CF01F6D22C20616BAF
:100570007469766965727400FC018894089501E2DB
:1005800022273581D7DE50F0CF01E6D22C207281B0
:10059000636B67657365747A7400FC010895DCD23F
:1005A00020676566756E64656E00089517E021E04A
:1005B00032E0CF0184DF98F4FC0131E080DF78F491
:1005C000FC0118E026E030E57ADFA8F5C5D24B65DE
:1005D000696E20447275636B6572210030C2CF0171
:1005E000BBD2447275636B657200D9DFFC0183DF97
:1005F000C8F0F0936900E0936800A9DF98F012E07A
:10060000BEDF6869B2E0A0E04D015D0108EF04BB08
:10061000AF9886D03CD16F7E9FD22C204F4B2E00BE
:100620000ED2089599D2202D204665686C657221FE
:10063000000005D20895CF018FD24D617373656EAE
:1006400073706569636865720000A9DFFC0153DFA0
:1006500048F300916B00013028F3F0936900E093B8
:1006600068001FEF8CDF6064CEE7F3E0EDE31FE08E
:10067000059109931A95E1F7CFCF5553424311479E
:100680001508000200008000100008DD61FF0895D9
:10069000F1E0EAEA91E080E0D2930197E9F785DEA4
:1006A00048F0F0E0EAEA6BD0F0E0EAEA7FDF67FDCD
:1006B0006BC066FF979A08950DE014E021D2B1D285
:1006C00000D0BDD1AEC256D31BE628D2F5DF0DE077
:1006D00014E016D2B2E0A0E09D918D9102970D91A9
:1006E000A4D10197E1F741C31DE0A5DC06FF089501
:1006F000CEDC32D22044657461636800A0D167FF0C
:1007000009C038D31BE60AD20CE013E0F9D189D234
:10071000D3DF2BD36627D4BBC5BA979AD7BB08952E
:10072000E0916800F091690001EA11E020E030E01A
:10073000458150E090E081E0B0E0ACE617DEA0F04B
:10074000892B91F40C9108731F2D177C102BF12E1F
:1007500013FDAB9A13FFAB9814FDAC9A14FFAC9841
:1007600015FDAD9A15FFAD9808951781110F165F0D
:100770005BD1019168D11A95D9F70895F6DF5FD161
:1007800000810023D9F70895F5D21BE6C7D10CE00C
:1007900013E0B6D1E0916800F0916900E6DFE5D2A0
:1007A000089564FD0895D501ED92BB7FB2605D01AF
:1007B000A825B925BA2B19F0AF98AE9A01C060618F
:1007C000677D0F920090720003940092720089F48A
:1007D0000090730003940092730059F40090740029
:1007E00003940092740029F4009075000394009221
:1007F0007500A0917600A068A09376000F90AF9945
:10080000D0CF089563FD0895D401C5018A1B9B0BC9
:1008100064FF20F494E080E08A1B9B0B80349D07EA
:1008200038F400916D000A9529F000936D00089549
:1008300080E49D2F0AE000936D00E0916800F09144
:10084000690020916A0040E18F93979A8FDC979816
:100850008F91E0F0BB7FB2604D0164FF03C0AF98A1
:10086000AE9A6F7EAA25BB25BA2B09F46860CEE646
:1008700014E088940881081F099388271A95D1F7F6
:1008800000E810917600102B109376000895E09107
:100890006800F091690001EA10E024812A9530E0B7
:1008A0004681558192E080E05FDD58F09D918D9109
:1008B000039738F00296923020F4606204DF889447
:1008C00008950894089501D0E0F00295102F159531
:1008D0001764F2E4E6EF31979A9B10C09899D9F724
:1008E00069F01F7B15BBF2E4E6EF31979A9B06C0D7
:1008F000989BD9F719F017E515BB089503B3A3D05A
:100900000894089563FF089516B303B30770063083
:10091000C1F7606165FD02C0BADF98F3FF920FEB8B
:10092000F02E0FE305BBF2E4E6EF31979A9B13C07C
:10093000AF9BD9F781F00E2D011769F4F2E4E6EFD1
:1009400031979A9B08C0829BD9F729F0AF9803B3DF
:100950000095077039F0FF906F7E0F2D0F770064C0
:1009600005BB089507E5143009F00F7E05BB07E4C9
:10097000F02E65D0F1D049454545313238343A47FB
:10098000657444657649645B0000012F5CD00DE519
:100990004CD0AC990CC0E0D0202D206E69636874F7
:1009A00020756E746572737481747A742100AC9BC7
:1009B00013C0B2E0A2E08E919E910D9184DF58F0B9
:1009C0000197D9F7C9D0204162686F6C756E6720B6
:1009D0004F4B2E0001C0AC98F0E0E0E001979A99EF
:1009E000E9F72DD0B8CFD098D89800EC07B906EC2D
:1009F00006B93699FECF369A3699FECF04B115B1B5
:100A000016950795D6B9D7B9D09A089567FF089576
:100A1000AF9B0895AF93BF930F930FB7C2DE0FBF85
:100A20000F91BF91AF91089500E2F0DF5D9BFDCF84
:100A30000CB90895EBDF5F9BFDCF7CB108950DE00D
:100A4000F4DF0AE0F2CF0F93029501D00F910F70FF
:100A5000005D0A3350F3095FE8CF11272F93112768
:100A600028E0000F111F1A3010F01A5003952A9534
:100A7000C1F72F9108952F9321E00A3028F0EDDF80
:100A80001F932395FACF0F910063CFDF2A95D9F7F3
:100A90002F910895CFDF7030E9F37B3109F008958D
:100AA000C9DF7B35E9F37F34D9F37B3103E0C1F053
:100AB000783401E0A9F07B3405E091F0713400E175
:100AC00079F072340EE061F0733406E049F074346A
:100AD00002E031F07035F8F27435E8F67C5608958E
:100AE000702F08950BE3A1CF0BE19FDF0BE59DCFA6
:100AF00000E29BCF0F3711F0003208F40FE595CFDD
:100B00000F93F2DF012F0395B6DFECDF0F91039512
:100B1000B2DF08E48ACF0770006387CFE5DF00E328
:100B200013FD039582DFDEDF03E37FDF012FF3DFB9
:100B3000D9DF04E37ADF012F02950770005D75DFCE
:100B400017FF03C0CFDF05E370DF0DE66ECF6DDF6B
:100B500005910023E1F70895FF91EF91EE0FFF1F3C
:100B6000F7DF3196F695E7950994219400E00309A3
:100B7000302E00E00409402E00E00509502E0895B3
:100B80002F93002720E2220C331C441C551C001F0D
:100B900010F0011710F0011B23942A95A1F72F9153
:100BA0000895022D0329042905290895332720E8F3
:100BB0001AE0122E2F700FE757FE1022002417FCA8
:100BC000D4DFDEDF005D0A3308F0095F0F93039482
:100BD0002A9529F416FC04C00CE20F9303948AF7BB
:100BE000E0DF79F70DE217FC03C00BE214FE02C050
:100BF0000F93039415FE08D00F9117DF15FC3A955B
:100C00000A94D1F715FE089530192AF021F000E278
:100C10000CDF3A95E1F708950F9380DF1F910027CD
:100C20006FDF1BE461DF012F00CF8901F5DF239522
:100C3000089517E073DF90DF1B5B324A000020E06D
:100C400030E7F3DF89DF204C505432555342202DDA
:100C5000204B6F6E76657274657220706172616C84
:100C60006C656C202D3E205553422D447275636B8C
:100C7000657220206823730037E6D7DF2C30E9F750
:100C800000E012E03DDF68DF204265747269656252
:100C9000737370616E6E756E673A09560D0A204463
:100CA00065736B726970746F723A0D0A2031323855
:100CB000342044657649443A0D0A0A0A2053746187
:100CC0007475733A201B5B346D4552521B5B323492
:100CD0006D3D58204F4E4C3D582050453D58201BEF
:100CE0005B346D41434B1B5B32346D3D58204253A6
:100CF000593D0D0A20476573656E646574652F451F
:100D00006D7066616E67656E652042797465733AD1
:100D1000090909092F0920206B427974652F730D89
:100D20000A0027E130E781DF17DF204669726D771F
:100D30006172652D45727374656C6C756E673A20CF
:100D400032372E30382E30362031343A30353A3082
:100D5000300017E0E3DE00DF1B5B31333B323372E0
:100D60001B5B31333B304800089515E75BDF17E02C
:100D7000D5DE089513E756DF0895299039904990FC
:100D8000599014CF23E05524220C331C441C551CCD
:100D9000220C331C441C551C38E00ACF03E112E03E
:100DA000AFDE21DE18014424552422E034E000DFC8
:100DB00005B310917700011779F1009377000DE0EA
:100DC00017E09EDE0CE4AB9908E4A39B0AE52DDE58
:100DD00003E117E095DE0CE4AC9908E4A49B0AE576
:100DE00024DE08E117E08CDE0CE4AD9908E4A59B55
:100DF0000AE51BDE0EE117E083DE0CE4AE9908E4A1
:100E0000A69B0AE512DE04E217E07ADE0CE4AF9955
:100E100008E4A79B0AE509DE4091760047FF0CC075
:100E20000DE118E06DDECEE6A8DF17E677DE0FE213
:100E3000FCDD1BE673DEA1DFCEE6B0E0A8E71127FC
:100E400029900C912D92201A39900C913D92300AE4
:100E500049900C914D92400A09F01064C395699035
:100E60000C916D92601A79900C917D92700A1880A5
:100E70000C911C92100A09F01064012F042B0074CD
:100E800071F04F7B16FD406400E318E039DE1F92DD
:100E900079DF4F90130113E4C5DE23E274DF4F774F
:100EA0004093760008952D5C7C2F14E737DE0FE425
:100EB00010E026DE0091760003950B7F009376000C
:100EC0000370FEE0E6EAE00FFD1F0491AECD04E002
:100ED0000EBF0FE50DBFDD2766270FEFC02E0BEB12
:100EE0000CBF0BE003BFCABAC5BA05EE02BB0AEFDE
:100EF00001BB02E005BF00E40BBF07EB0BBD0AE13D
:100F00000ABD0BE00EBD0027F0E0E0E694E080E0D3
:100F100001930197E9F7789400E000BD03E109B976
:100F200008E10AB905E9F02EB2D804E66ED881DEF0
:100F300000EC00937600D093770067FF03C024DCB9
:100F400065FDC1DB67FF03C05DDCDCDCE9DB61FF65
:100F50009CDB61FDC9DB08B704FF08C000E108BFE6
:100F600009DFA3DF1BE6DADD19DFFFDE5F9BEACFD7
:100F700091DD7C30E1F2723111F4F894A8CF703732
:100F800021F48A9A92988A98929A743669F467FF43
:100F900008C063FF06C0AF9A606179DC6F7EAF98CE
:100FA00088F607E042DDCECF753639F4D5DD457AD7
:100FB000426974733D00062F46DD7936E9F43FDD62
:100FC000CBDD496E666F3A203C34303E2C3C3432E7
:100FD0003E3D4E414B2C203C38303E3D5354414C1D
:100FE0004C2C203C31303E3D446973636F6E6E651E
:100FF00063742E2E2E0023DD7237E9F4CEE6002432
:101000000992099209920992099209920992099208
:10101000C8E709920992099209920992099230DC73
:10102000A9DE1BE67BDD0DE118E06ADD12E1FCDCE8
:081030001A95E9F79ADE86CF5C
:00000001FF
